:020000040000FA
:1000000000306500FF30660090019101920193017C
:100010009401970140309800803099001008120236
:10002000031C1528851405121728851005161008BD
:100030001302031C1D2805151E28051110081402A3
:10004000031C2428851525288511900A03192920C9
:100050000E28910A111C970A170895003B20920060
:100060001808170795003B209300190817079500FB
:100070003B209400080080309600150816020318F3
:0E00800045289600803016020800150808007A
:02400E00F23F7F
:00000001FF
